:100000000C9437050C9480050C9485060C9480059F
:100010000C9480050C9480050C9480050C9480054C
:100020000C9480050C9480050C946F0D0C94450E77
:100030000C94341D0C9480050C9480050C94800560
:100040000C9480050C9480050C9480050C9480051C
:100050000C9480050C94A81D0C9480050C948005CC
:100060000C9480050C9480050C9480050C948005FC
:100070000C9480050C9480050C9480050C948005EC
:100080000C9480050C9480050C9480050C948005DC
:100090000C9480050C948005A407B707D007D407FB
:1000A000D807DB07E107E507E907ED07F107B60E1B
:1000B000D80EC60FD80EC60F1D0F400FC60F950FD6
:1000C000A80FFD12FD122C132C138A13C813E2156E
:1000D000E215E113E215E214E214B615E215E21599
:1000E000CD1500291E1F20212223242526272D2E51
:1000F0002A2B141A0815171C180C12132F3028E07D
:10010000041607090A0B0D0E0F333435E1311D1BA0
:100110000619051110363738E555E22C393A3B3CC3
:100120003D3E3F4041424353475F6061565C5D5EE8
:1001300057595A5B626358E4544445E6ABE3E765BC
:10014000A5A6A8B4B0A7AFB6BCBBBAB9B8B5B3B290
:10015000AC4A524BAA50A94FB74D514E494C464854
:100160000000706275663A2066756C6C0A00253076
:10017000325820004B6579626F617264207374613C
:1001800072742E0A0055534220636F6E666967755C
:100190007265642E0A000D0A696E69740A005B4478
:1001A0005D005B435D002C035800540020006B0091
:1001B0006500790062006F00610072006400200039
:1001C00063006F006E0076006500720074006500C9
:1001D000720000000E0374002E006D002E006B00F4
:1001E0002E0000000403090409028D00050100A08F
:1001F000320904000001030101000921110100017D
:100200002240000705810308000A090401000103D8
:10021000010200092111010001224D00070582039E
:1002200008000A090402000103000000092111016D
:1002300000012236000705830308000A09040300B1
:10024000020300000009211101000122220007051C
:1002500084032000010705040320000109040400B1
:1002600001030000000921110100012239000705E6
:1002700085032000011201100100000008EDFE12AC
:100280006501000102000105010906A10105071928
:10029000E029E71500250195087501810205081977
:1002A00001290595057501910295017503910105D7
:1002B00007190029F71500250195F875018102C07D
:1002C0000631FF0974A1010975150026FF0095206C
:1002D000750881020976150026FF009520750891A2
:1002E00002C005010980A101850216810026B70020
:1002F0001A81002AB700751095018100C0050C090C
:1003000001A1018503160100269C021A01002A9C06
:1003100002751095018100C005010902A1010901C2
:10032000A10005091901290515002501950575018B
:10033000810295017503810105010930093115819B
:10034000257F95027508810609381581257F95015D
:1003500075088106050C0A38021581257F950175FF
:10036000088106C0C005010906A101050719E02999
:10037000E715002501950875018102950175088131
:100380000105081901290595057501910295017569
:100390000391010507190029FF150026FF009506A6
:1003A00075088100C0636F6E73756D65723A2025A4
:1003B0003034580A0073797374656D3A20253034EF
:1003C000580A000A002530325820006B6579626FA8
:1003D0006172643A20004C45443A20253032580A74
:1003E00000253032583A202530386225730A0072D1
:1003F0002F632030313233343536370A0064656C70
:100400005F6B65795F6269743A2063616E2774205F
:1004100064656C3A20253032580A006164645F6B71
:1004200065795F6269743A2063616E277420616444
:10043000643A20253032580A00290A002575002F19
:10044000002575005D28002564002000256400203B
:100450000025640020002564007C0025303258000F
:100460006D6F7573656B6579205B62746E7C782047
:1004700079207620685D287265702F61636C293A57
:10048000205B006D6B5F776865656C5F74696D6597
:100490005F746F5F6D6178203D2025640A006D6B8D
:1004A0005F776865656C5F6D61785F7370656564C3
:1004B000203D2025640A006D6B5F74696D655F7473
:1004C0006F5F6D6178203D2025640A006D6B5F6D64
:1004D00061785F7370656564203D2025640A006D56
:1004E0006B5F696E74657276616C203D2025640ACD
:1004F000006D6B5F64656C6179203D2025640A00A6
:100500006D6B5F776865656C5F74696D655F746F4F
:100510005F6D6178203D2025640A006D6B5F776810
:1005200065656C5F6D61785F7370656564203D2003
:1005300025640A006D6B5F74696D655F746F5F6D34
:100540006178203D2025640A006D6B5F6D61785FE6
:100550007370656564203D2025640A006D6B5F69DA
:100560006E74657276616C203D2025640A006D6BA7
:100570005F64656C6179203D2025640A000A0025CE
:100580007500363A20776865656C5F74696D655FE4
:10059000746F5F6D61783A20000A00257500353A66
:1005A00020776865656C5F6D61785F737065656401
:1005B0003A20000A00257500343A2074696D655FA1
:1005C000746F5F6D61783A20000A00257500333A38
:1005D000206D61785F73706565643A20000A0025BC
:1005E0007500323A20696E74657276616C286D739D
:1005F000293A20000A00257500313A2064656C61B3
:1006000079282A31306D73293A20000A092D2056A5
:10061000616C756573202D0A004D3E004D25643ECA
:1006200020003F007365742064656661756C740A10
:1006300000433E200077686572652064656C7461D4
:100640003A20637572736F723D25642C207768655C
:10065000656C3D25640A53656520687474703A2F93
:100660002F656E2E77696B6970656469612E6F7294
:10067000672F77696B692F4D6F7573655F6B657950
:10068000730A000A092D204D6F7573656B6579201B
:100690002D0A4553432F713A09717569740A313A2D
:1006A0000964656C6179282A31306D73290A323A00
:1006B00009696E74657276616C286D73290A333A24
:1006C000096D61785F73706565640A343A0974690D
:1006D0006D655F746F5F6D61780A353A097768659B
:1006E000656C5F6D61785F73706565640A363A09A1
:1006F000776865656C5F74696D655F746F5F6D6168
:10070000780A0A703A097072696E742076616C75A5
:1007100065730A643A097365742064656661756C73
:1007200074730A75703A092B310A646F776E3A094F
:100730002D310A706775703A092B31300A70676481
:100740006F776E3A092D31300A0A7370656564203F
:100750003D2064656C7461202A206D61785F737040
:10076000656564202A2028726570656174202F20D9
:1007700074696D655F746F5F6D6178290A003F0071
:100780004D3E2000433E20004C25640A000A092DFE
:1007900020436F6E736F6C65202D0A4553432F7194
:1007A0003A09717569740A6D3A096D6F7573656BF5
:1007B00065790A000A092D204D61676963202D0AB9
:1007C000643A0964656275670A783A096465627516
:1007D00067206D61747269780A6B3A0964656275A5
:1007E00067206B6579626F6172640A6D3A096465AE
:1007F000627567206D6F7573650A763A0976657262
:1008000073696F6E0A733A097374617475730A635E
:100810003A09636F6E736F6C65206D6F64650A30A3
:100820002D343A096C61796572302D3428463130A7
:100830002D4634290A506175733A09626F6F746CE2
:100840006F616465720A6E3A094E4B524F0A003F5F
:10085000004E4B524F3A206F66660A004E4B524F85
:100860003A206F6E0A0074696D65725F726561642B
:10087000333228293A202530346C580A006B6579C8
:10088000626F6172645F6E6B726F3A2025580A0066
:100890006B6579626F6172645F69646C653A20258B
:1008A000580A006B6579626F6172645F70726F7471
:1008B0006F636F6C3A2025580A00686F73745F6B22
:1008C0006579626F6172645F6C65647328293A2090
:1008D00025580A000A092D20537461747573202D60
:1008E0000A004743433A20342E392E3220415652D3
:1008F0002D4C4942433A20312E382E3073766E20EB
:100900004156525F415243483A2061767235310A6E
:10091000004F5054494F4E533A204C554641204DBC
:100920004F5553454B45592045585452414B455915
:1009300020434F4E534F4C4520434F4D4D414E4465
:10094000204E4B524F203531320A004255494C441B
:100950003A20343630616139302D646972747920FF
:100960002830363A35393A3332204D6172203135EC
:100970002032303138290A005649443A203078462E
:1009800045454428742E6D2E6B2E29205049443A3B
:1009900020307836353132285854206B6579626FB3
:1009A00061726420636F6E76657274657229205679
:1009B00045523A203078303030310A0044455343B4
:1009C0003A20636F6E76657274205854206B657997
:1009D000626F61726420746F205553420A000A09E5
:1009E0002D2056657273696F6E202D0A000A6D6F97
:1009F0007573653A206F66660A000A6D6F757365D8
:100A00003A206F6E0A000A6B6579626F6172643A10
:100A1000206F66660A000A6B6579626F6172643ADC
:100A2000206F6E0A000A6D61747269783A206F66F1
:100A3000660A000A6D61747269783A206F6E0A0066
:100A40000A64656275673A206F6E0A000A6465621F
:100A500075673A206F66660A000A0A626F6F746CE7
:100A60006F616465722E2E2E2000433E20001124FB
:100A70001FBECFEFD0E2DEBFCDBF04B603FE27C05E
:100A80008091CF029091D002A091D102B091D20278
:100A90008730904BA740B04BD1F41092CF02109208
:100AA000D0021092D1021092D20214BE84B7877F76
:100AB00084BF0FB6F894A8958091600088618093F8
:100AC0006000109260000FBEE0E0FFEF099511E0BA
:100AD000A0E0B1E0E0EAFDE400E00BBF02C0079057
:100AE0000D92A833B107D9F722E0A8E3B1E001C025
:100AF0001D92AF3CB207E1F70E94930A0C94CE26F8
:100B00000C940000FF93EF93E0913801F0913901CC
:100B1000309709F00995EF91FF910895FC018591B7
:100B2000803011F0EFDFFBCF0895FF27E0E230E2E5
:100B300047FF0CC0419597FF09C0EDE260957095A5
:100B400080959095611D711D811D911D27FF02C02B
:100B5000219530E350E2AA27660F771F881F991F5F
:100B6000AA1FA41710F0A41B63955A95A9F7AA30E1
:100B700008F0A95FA05DAF93F3956115710581053C
:100B8000910541F7ED3211F4EF93F395F21718F454
:100B90003F93F395FBCF8F91B5DFFA95E1F7089579
:100BA000E991F9918591803021F0853219F0AADF21
:100BB000F9CF089520E0E89455915532C1F35033B0
:100BC00011F4689455915A3348F4505390F3220F1E
:100BD000022E220F220F200D250FF4CF0EF42195A7
:100BE00089919991533619F3533729F1533559F1B6
:100BF000BC0188279927E8945C3621F48991999162
:100C000068945591543639F446EF7EF077FF0DC065
:100C10008FEF9FEF0AC055374AE039F0583540E171
:100C200021F0523642E009F00895FF93EF937DDF03
:100C3000EF91FF91B7CFFF93EF93FC01819180304B
:100C4000B9F360DFFBCFFF93EF9368DFF1CFDF9362
:100C5000CF93CDB7DEB72596A3DFCF91DF9108956F
:100C6000E9E6F0E0808188608083E9982F98279AF0
:100C70002FEF89E698E1215080409040E1F700C0D5
:100C8000000027985898509A5998519A2FEF89EF59
:100C900090E0215080409040E1F700C00000519862
:100CA000599A5098589AE19AE99A08954FB7F8944A
:100CB00020913E0130913F0180913C0190913D0196
:100CC0004FBF28173907F9F09FB7F89420913C01DE
:100CD00030913D0140913E0150913F014217530731
:100CE00079F0F901EE0FFF1FE05CFE4F80812F5F6E
:100CF0003F4F2F71332730933D0120933C0101C0BA
:100D000080E09FBF089580E008951F920F920FB674
:100D10000F9211240BB60F922F933F934F935F9333
:100D20006F937F938F939F93AF93BF93CF93EF93E3
:100D3000FF9329B1217090913B01992319F09930CB
:100D400058F403C0211108C037C080913A0186953C
:100D50002111806880933A0181E0890F80933B01E3
:100D6000983051F540913A0150E0CFB7F894809116
:100D70003E0190913F019C012F5F3F4F2F71332720
:100D800060913C0170913D012617370761F0880F93
:100D9000991FFC01E05CFE4F5183408330933F017B
:100DA00020933E0104C082E691E00E948E05CFBFF1
:100DB00010923B0110923A01FF91EF91CF91BF91B8
:100DC000AF919F918F917F916F915F914F913F91E3
:100DD0002F910F900BBE0F900FBE0F901F90189584
:100DE000803389F1A0F48E3138F48C3140F58031B4
:100DF00081F1893111F10895843219F128F490EECE
:100E0000980F9330F0F008958E32E9F008958A3407
:100E100048F48734E0F48533C1F08833B1F082338D
:100E2000C9F411C08D3499F018F48B3481F0089511
:100E300091EB980F953058F008958AE50895885CF5
:100E40000895805C08958C5B08958F5D0895885D9A
:100E500008958EE60895CF93DF93D82FD770C82FCB
:100E6000C695C695C6956D2F8C2F0E944B11882371
:100E700071F0EC2FF0E0EF57FE4F81E090E001C001
:100E8000880FDA95EAF78095908189238083DF9136
:100E9000CF910895CF93DF93D82FD770C82FC695E1
:100EA000C695C6956D2F8C2F0E944B1181110DC0D8
:100EB000EC2FF0E0EF57FE4F81E090E001C0880F8B
:100EC000DA95EAF79081892B8083DF91CF9108959D
:100ED0008091B10281608093B1020E943006E1E806
:100EE000F1E080E18E0F11928E13FDCF0895CF9324
:100EF000DF931F92CDB7DEB765E08FE00E944B1104
:100F0000882319F08DE70E942B070E94560688233C
:100F100071F01F928F932EE631E03F932F938983D8
:100F20000E9427060F900F900F900F908981E091FB
:100F300080014E2F50E04B30510508F058C0FA01A7
:100F4000E45BFF4F0C94B126803E21F0813E21F4FA
:100F500086E014C081E012C01816BCF09FE7980F1D
:100F60009E3708F044C080580E942B0740C08A3248
:100F700021F0873B31F484E001C082E0809380015E
:100F800038C018162CF40E94F0060E944A072FC0A1
:100F90009FE7980F9E3758F580580E94F006E4CFDF
:100FA000803E29F583E0EACF873309F58CE71CC042
:100FB000803EE9F41EC08A3AD1F48CE70E942B07E8
:100FC00018C08D31A1F487E0D9CF853481F488E051
:100FD000D5CF813E61F489E0D1CF8D3941F48AE0EB
:100FE000CDCF853C21F48DE70E944A0702C01092C4
:100FF000800181E00F90DF91CF910895E82FF0E01C
:10100000EF57FE4F80810895E1E8F1E080E18E0F17
:1010100011928E13FDCF089508958091B501089522
:101020009FB7F894109294019FBF9091C60294309C
:1010300009F057C09091E9009F703091EC00232F88
:10104000217030FD20E8922B24E02093E9002091CC
:10105000EB0020FF43C02091EE0027FF3FC020910E
:101060009101222321F02091E80025FF37C0109242
:10107000910126E03091E80035FD15C03091C6029F
:10108000343061F53091EB0035FD28C0215021F45A
:1010900081E08093910122C0EFE9FFE03197F1F701
:1010A00000C00000E7CF8093F1008091E80085FD4B
:1010B0000AC08091E80080FFFCCF8091E8008E7725
:1010C0008093E80006C08FB7F89421E02093940144
:1010D0008FBF9F709093E90080E008959F70909378
:1010E000E9008FEF0895CF93DF9300D01F92CDB723
:1010F000DEB79C018091C602843019F593E0998394
:101100003B832A839093E9008FEF9091E800815010
:1011100095FD06C095ED9A95F1F700008111F5CF88
:101120008091E80085FF0DC040E050E063E070E092
:10113000CE0101960E94600B8091E8008E7780932B
:10114000E8000F900F900F90DF91CF910895CF930B
:10115000DF9300D01F92CDB7DEB72091C6022430B6
:1011600021F522E029839B838A8383E08093E90031
:101170008FEF9091E800815095FD06C095ED9A950E
:10118000F1F700008111F5CF8091E80085FF0DC0D7
:1011900040E050E063E070E0CE0101960E94600BF9
:1011A0008091E8008E778093E8000F900F900F9069
:1011B000DF91CF9108952091C6022430F1F422E00E
:1011C0002093E9002FEF3091E800215035FD06C053
:1011D00035ED3A95F1F700002111F5CF2091E800A7
:1011E00025FF0BC040E050E065E070E00E94600B1E
:1011F0008091E8008E778093E8000895CF93DF9385
:101200002091C602243009F048C0EC0180910A0107
:101210008823E1F080910B018823C1F085E0809361
:10122000E9008FEF9091E800815095FD06C09AE2A9
:101230009A95F1F700C08111F5CF8091E80085FF04
:101240002CC040E050E060E270E017C081E0809385
:10125000E9008FEF9091E800815095FD06C095ED73
:101260009A95F1F700008111F5CF8091E80085FF94
:1012700014C040E050E068E070E0CE010E94600BD6
:101280008091E8008E778093E80080E2FE01A5E976
:10129000B1E001900D928A95E1F7DF91CF91089529
:1012A00082EA91E00E948E058091C502811109C0F9
:1012B0000E94F10C0E94530D8091E20084608093A3
:1012C000E20008958EE991E00E948E051092C50219
:1012D00008950895209192012F5F822F62E30E946A
:1012E0009126992319F0209392010895109292016A
:1012F00080919401882371F18091C602843041F578
:101300008091E9008F702091EC00922F917020FD68
:1013100090E8892B94E09093E9009091EB0090FF86
:1013200014C09091EE0097FF10C09091E80095FFD7
:1013300003C01092F100F9CF9091E80090FF05C032
:101340009091E8009E779093E8008F708093E90079
:1013500010929401089542E061EC81E00E946B0CD0
:1013600042E061EC82E00E946B0C42E061EC83E0C1
:101370000E946B0C42E261EC84E00E946B0C42E242
:1013800061EC85E00C946B0C8091C802833009F409
:1013900055C030F4813071F0823009F48EC0089568
:1013A0008A3009F47AC08B3009F460C0893009F0C2
:1013B0009CC020C08091C702813A09F096C08091FC
:1013C000E800877F8093E8008091CB029091CC0267
:1013D000892B21F460E285E991E003C060E080E0C0
:1013E00090E070E00E94AB0B8091E8008B778093D7
:1013F000E80008958091C702813209F076C080919B
:10140000CB029091CC02009719F0049709F06DC0BF
:101410008091E800877F8093E8008091E80082FD5A
:1014200005C08091C6028111F8CF5FC08091F100A4
:101430008093B5018091E8008B7753C08091C702FB
:10144000813A09F052C08091CB029091CC02892B55
:1014500009F04BC08091E800877F8093E80080917D
:10146000E80080FFFCCF80910A0136C08091C7025E
:101470008132D9F58091CB029091CC02892BA9F5CC
:101480008091E800877F8093E8000E94A00C809103
:10149000C90280930A010C9404168091C70281321C
:1014A00021F58091E800877F8093E8000E94A00CDE
:1014B0008091CA028093B60108958091C702813A53
:1014C000A1F48091E800877F8093E8008091E80094
:1014D00080FFFCCF8091B6018093F1008091E800FD
:1014E0008E778093E8000C94A00C089508950895D9
:1014F0008091B501809393011092B50180E00E9424
:101500000C080E9404080C9404160C94780A0E949B
:10151000F31C8091C402882329F00E941C1D8111B4
:101520000C944A0B089584B7877F84BF0FB6F89454
:10153000A89580916000886180936000109260009F
:101540000FBE90E080E80FB6F8948093610090930E
:1015500061000FBE80E198E00E94C41C86E991E022
:101560000E948E050E94760A0E949F100E94F10C34
:101570000E94530D8091E20084608093E200789491
:101580008091C6028430E1F781ED97E0019739F050
:10159000EFE9FFE03197F1F700C00000F7CF85E8F1
:1015A00091E00E948E050E94A11080E091E00E94CF
:1015B000DE0F84E791E00E948E050E94770A8091F9
:1015C000C602853019F40E94870AF9CF0E94A5103F
:1015D000F6CF0E94301D809193018093B50108954C
:1015E0000C94E90A292F332723303105C9F064F41C
:1015F0002130310581F02230310509F043C08DE8FA
:1016000090E028EE31E042C021323105F1F0223283
:10161000310541F137C082E190E025E732E036C084
:1016200099278130910541F08230910541F0892B55
:1016300049F5E4EEF1E005C0E4EDF1E002C0E6EAD0
:10164000F1E0849190E09F0121C06530D8F4E62F4D
:10165000F0E0EE0FFF1FED5DFE4F2081318189E04C
:1016600090E014C0653070F470E0FB01EE0FFF1FD6
:10167000E75EFE4F20813181FB01EC5EFE4F8081F1
:1016800090E004C080E090E020E030E0FA01318397
:101690002083089584E189BD86E189BD09B400FEF7
:1016A000FDCF8091D8008F7D8093D8008091E0009D
:1016B00082608093E0008091E00081FDFCCF08957E
:1016C000CF92DF92EF92FF920F931F93CF93DF930E
:1016D000EC018B016A010E94BF0C811133C0C1145F
:1016E000D10439F0F60180819181081B190BC80FD4
:1016F000D91FE12CF12C0115110519F18091E80099
:1017000085FD16C08091E8008E778093E800C114B3
:10171000D10449F0F60180819181E80EF91EF18231
:10172000E08285E00FC00E94BF0C882321F30AC02D
:1017300089918093F10001501109FFEFEF1AFF0A20
:10174000DACF80E0DF91CF911F910F91FF90EF9062
:10175000DF90CF9008952091CD023091CE022617D0
:10176000370748F06115710539F42091E8002E77AC
:101770002093E80001C0B90140E06115710599F1BD
:101780002091C602222309F441C0253009F440C04B
:101790002091E80023FD3EC02091E80022FD30C0EA
:1017A0002091E80020FFE9CF2091F2003091F30072
:1017B000FC01CF016115710559F02830310540F465
:1017C00081918093F100615071092F5F3F4FF1CFFC
:1017D00041E02830310509F040E02091E8002E7703
:1017E0002093E800CACF4111CBCF0AC08091C60236
:1017F000882361F0853061F08091E80083FD0AC0A4
:101800008091E80082FFF2CF80E0089582E00895A1
:1018100083E0089581E008952091CD023091CE02B9
:101820002617370748F06115710539F42091E80053
:101830002E772093E80001C0B901FC0120E061157A
:10184000710581F18091C602882309F43EC085307C
:1018500009F43DC08091E80083FD3BC08091E80021
:1018600082FD2DC08091E80080FFE9CF8091F200D9
:101870009091F3006115710559F08830910540F49D
:1018800024912093F1003196615071090196F2CFB5
:1018900021E0089709F020E08091E8008E7780939E
:1018A000E800CDCF2111CECF0AC08091C602882397
:1018B00061F0853061F08091E80083FD0AC080917D
:1018C000E80082FFF2CF80E0089582E0089583E08F
:1018D000089581E00895982F973058F59093E90086
:1018E000981739F07091EC002091ED005091F000C4
:1018F00003C0242F762F50E021FF19C03091EB0058
:101900003E7F3093EB003091ED003D7F3093ED0052
:101910003091EB0031603093EB007093EC0020933A
:10192000ED005093F0002091EE0027FF07C09F5F6D
:10193000D3CF8F708093E90081E0089580E008950F
:101940008091C70287FF11C08091E80082FD05C029
:101950008091C6028111F8CF11C08091E8008B7789
:101960000BC08091C602882349F08091E80080FF77
:10197000F8CF8091E8008E778093E8000895209159
:10198000E4003091E50095E64091EC00842F8170F1
:1019900040FF22C08091E80080FD1CC08091C602FB
:1019A000882391F0853091F08091EB0085FD10C087
:1019B0004091E4005091E5004217530729F39A0142
:1019C000915011F784E0089582E0089583E008952E
:1019D00081E0089580E008954091E80042FFDECF65
:1019E00008950E94620D0E946A0DE0EEF0E0808191
:1019F00081608083E8EDF0E080818F77808319BC7F
:101A0000A7EDB0E08C918E7F8C9380818F7E808358
:101A10001092C50208950F931F93CF93DF930E94F6
:101A2000620D0E946A0DC8EDD0E088818F778883AF
:101A300088818068888388818F7D8883E7EDF0E0E6
:101A400080818068808319BC1092C6021092C20205
:101A50001092C4021092C30200EE10E0F8018081DF
:101A60008B7F808388818160888342E060E080E0B2
:101A70000E946B0CE1EEF0E080818E7F8083E2EECD
:101A8000F0E0808181608083808188608083F801BC
:101A900080818E7F8083888180618883DF91CF9170
:101AA0001F910F910895E8EDF0E080818F7E808393
:101AB000E7EDF0E080818160808381E08093C50262
:101AC0000C940B0DE8EDF0E080818C7F8083109208
:101AD000E20008951092DA001092E10008951F923A
:101AE0000F920FB60F9211240BB60F922F933F93C4
:101AF0004F935F936F937F938F939F93AF93BF9316
:101B0000EF93FF938091E10082FF0BC08091E20090
:101B100082FF07C08091E1008B7F8093E1000E94EB
:101B20006A098091DA0080FF1FC08091D80080FF91
:101B30001BC08091DA008E7F8093DA008091D900FB
:101B400080FF0DC084E189BD86E189BD09B400FE36
:101B5000FDCF81E08093C6020E94500905C019BCE8
:101B60001092C6020E9462098091E10080FF19C0B4
:101B70008091E20080FF15C08091E2008E7F80930B
:101B8000E2008091E20080618093E2008091D800C1
:101B900080628093D80019BC85E08093C6020E94C1
:101BA000850A8091E10084FF30C08091E20084FFCB
:101BB0002CC084E189BD86E189BD09B400FEFDCF5A
:101BC0008091D8008F7D8093D8008091E1008F7E36
:101BD0008093E1008091E2008F7E8093E20080910B
:101BE000E20081608093E2008091C202882311F0BC
:101BF00084E007C08091E30087FD02C081E001C05E
:101C000083E08093C6020E94F00A8091E10083FF86
:101C100029C08091E20083FF25C08091E100877F89
:101C20008093E10082E08093C6021092C20280910C
:101C3000E1008E7F8093E1008091E2008E7F8093AF
:101C4000E2008091E20080618093E20042E060E087
:101C500080E00E946B0C8091F00088608093F0001F
:101C60000E946909FF91EF91BF91AF919F918F9170
:101C70007F916F915F914F913F912F910F900BBE8C
:101C80000F900FBE0F901F9018951F920F920FB6D6
:101C90000F9211240BB60F922F933F934F935F93A4
:101CA0006F937F938F939F93AF93BF93CF93DF9364
:101CB000EF93FF93C091E900CF708091EC00D82F93
:101CC000D17080FDD0E81092E9008091F000877F0C
:101CD0008093F00078940E948D0E1092E90080911C
:101CE000F00088608093F000CD2BCF70C093E900A6
:101CF000FF91EF91DF91CF91BF91AF919F918F9124
:101D00007F916F915F914F913F912F910F900BBEFB
:101D10000F900FBE0F901F9018951F93CF93DF93D6
:101D2000CDB7DEB7AA970FB6F894DEBF0FBECDBF12
:101D3000E7ECF2E088E08E0F9091F10091938E1322
:101D4000FBCF0E94C4098091E80083FF1FC18091EE
:101D5000C7029091C802492F50E04A30510508F05F
:101D600015C1FA01E95AFF4F0C94B126803881F071
:101D7000823809F00BC18091CB028F708093E9000B
:101D80008091EB0085FB882780F91092E90006C05E
:101D90008091C3029091C402911182609091E800F9
:101DA000977F9093E8008093F1001092F100C8C0F3
:101DB000282F2D7F09F0EAC0882319F0823061F0C6
:101DC000E5C08091C902813009F0E0C0933009F08C
:101DD00080E08093C4022BC08091C902811127C08A
:101DE0008091CB028F7009F4D1C08093E9002091DB
:101DF000EB0020FF1CC0933021F48091EB00806247
:101E000014C09091EB0090619093EB0021E030E0E2
:101E1000A90102C0440F551F8A95E2F74093EA00DA
:101E20001092EA008091EB0088608093EB001092A2
:101E3000E9008091E800877F86C08111A7C01091DA
:101E4000C9021F778091E3008078812B8093E300A3
:101E50008091E800877F8093E8000E94A00C809129
:101E6000E80080FFFCCF8091E30080688093E3006E
:101E7000111102C082E001C083E08093C60286C0D7
:101E80008058823008F082C08091C9029091CA02C5
:101E90008C3D53E0950779F583E08A838AE2898354
:101EA0004FB7F894DE01139620E03EE051E2E32FB5
:101EB000F0E050935700E49120FF03C0E295EF70EB
:101EC0003F5FEF708E2F90E0EA3010F0C79601C0B0
:101ED000C0968D939D932F5F243149F74FBF80911A
:101EE000E800877F8093E8006AE270E0CE01019607
:101EF0000E94AB0B14C0AE014F5F5F4F6091CB02ED
:101F00000E94F20ABC01892B09F440C09091E800BC
:101F1000977F9093E80089819A810E940C0C8091B0
:101F2000E8008B778093E80031C0803879F58091A4
:101F3000E800877F8093E8008091C2028093F100DF
:101F40008091E8008E778093E8000E94A00C1EC06C
:101F500081111CC09091C9029230C0F48091E800B8
:101F6000877F8093E8009093C2020E94A00C80912A
:101F7000C202811106C08091E30087FD02C081E0AA
:101F800001C084E08093C6020E94AB098091E80002
:101F900083FF0AC08091E800877F8093E8008091EA
:101FA000EB0080628093EB00AA960FB6F894DEBF38
:101FB0000FBECDBFDF91CF911F9108959093BC01CB
:101FC0008093BB010895E091BB01F091BC01309773
:101FD00021F00190F081E02D099480E00895EF92C6
:101FE000FF920F931F93CF93DF93E091BB01F0918A
:101FF000BC013097B1F18C010280F381E02D09958D
:102000008091B10282FF2DC080FF04C08BEC93E071
:102010000E948E05E80110E285ECE82E83E0F82EA0
:102020008091B10280FF0BC088811F928F93FF9235
:10203000EF920E9427060F900F900F900F90115073
:1020400021961111EDCF8091B10280FF0AC083EC7F
:1020500093E0DF91CF911F910F91FF90EF900C943F
:102060008E05DF91CF911F910F91FF90EF90089512
:10207000E091BB01F091BC01309721F00480F58123
:10208000E02D09940895CF93DF93EC018091B9017D
:102090009091BA01C817D90709F1D093BA01C0933A
:1020A000B901E091BB01F091BC013097B9F0068015
:1020B000F781E02DCE0109958091B10282FF0EC01B
:1020C00080FF0CC0DF93CF9385EB93E09F938F93BA
:1020D0000E9427060F900F900F900F90DF91CF91E5
:1020E0000895CF93DF93EC018091B7019091B801EF
:1020F000C817D90709F1D093B801C093B701E0918F
:10210000BB01F091BC013097B9F00084F185E02D5E
:10211000CE0109958091B10282FF0EC080FF0CC0F4
:10212000DF93CF9385EA93E09F938F930E942706D6
:102130000F900F900F900F90DF91CF9108950C9416
:102140004A110E945D1D0C946807BF92CF92DF92E6
:10215000EF92FF920F931F93CF93DF9300D000D0A5
:102160001F92CDB7DEB70E9477070EEB11E0F12C7E
:102170008F2D0E94FE07B82EF801C080C82639F4C2
:10218000F3940F5F1F4FF0E1FF12F2CF30C0809148
:10219000B10281FD0E946611D12CEE24E3948E2DB4
:1021A0008C21F9F0D982FA8281E09E2D9B2109F4DD
:1021B00080E08B830E94661D8160782F9D838C83D5
:1021C00049815A816B818D810E949C1149815A817C
:1021D0006B817C818D810E94E01CF80190819E259D
:1021E0009083D394EE0CF8E0DF12D9CFC9CF8FEFF4
:1021F00089838A831B820E94661D8160782F9D835C
:102200008C8349815A816B818D810E949C110E942F
:10221000DF1C0E94BF201091BD010E94E30F181720
:1022200041F10E94E30F8093BD019091B10292FFB2
:102230000EC090FF0CC01F928F9386ED93E09F938A
:102240008F930E9427060F900F900F900F90809110
:10225000BD010F900F900F900F900F90DF91CF91D5
:102260001F910F91FF90EF90DF90CF90BF900C9453
:10227000F11C0F900F900F900F900F90DF91CF9166
:102280001F910F91FF90EF90DF90CF90BF90089536
:102290000C940C080895CF93DF931F92CDB7DEB74F
:1022A00069830E94FE0790E021E030E0698102C06E
:1022B000220F331F6A95E2F72823392381E0232B6D
:1022C00009F480E00F90DF91CF910895EF92FF9293
:1022D0000F931F93CF93DF938FEE93E00E948E05B1
:1022E000C0E0D0E08DE2E82E81E0F82E01EE13E0B0
:1022F0008C2F0E94FE070E94C91CFF92EF921F9232
:102300008F93DF93CF931F930F930E9427062196FD
:102310008DB79EB708960FB6F8949EBF0FBE8DBFBF
:10232000C031D10529F7DF91CF911F910F91FF9017
:10233000EF90089508950895CF93DF93CDB7DEB75A
:102340002B970FB6F894DEBF0FBECDBF942F4F83EF
:10235000252F588769877A878B874A855B85452B28
:1023600021F02F3F09F59F3FF9F4DE01119686E039
:10237000FD0111928A95E9F785E0FE0137960190FB
:102380000D928A95E1F749815A816B817C818D811B
:102390009E810E94E1182B960FB6F894DEBF0FBE07
:1023A000CDBFDF91CF9108954F81588569857A859A
:1023B0008B850E94E01CD9CFCF93882309F4A4C059
:1023C000C82F8CEF8C0F813A48F48C2F0E9409247F
:1023D00081119AC08C2F0E94B91B0CC080E28C0F17
:1023E000883058F4C77081E001C0880FCA95EAF7B9
:1023F0000E94641CCF910C949E1C8BE58C0F833043
:1024000078F4C53A29F0C63A31F083E890E005C087
:1024100081E890E002C082E890E0CF910C944310F4
:1024200088E58C0F853108F06FC0C83A61F1C93A70
:1024300069F1CA3A71F1CB3A79F1CC3A81F1CD3AEE
:1024400089F1CE3A91F1CF3A99F1C13BA1F1C03B6C
:10245000A9F1C23BB1F1C33BB9F1C43BC1F1C53BEA
:10246000C9F1C63BD1F1C73BD9F1C83BE1F1C93B4A
:10247000E9F1CA3BF1F1CB3BF9F1CC3B09F43FC0A8
:1024800080E090E03EC082EE90E03BC089EE90E0BC
:1024900038C08AEE90E035C085EB90E032C086EB24
:1024A00090E02FC083EB90E02CC084EB90E029C03B
:1024B00087EB90E026C08CEC90E023C08DEC90E0A0
:1024C00020C083E891E01DC08AE891E01AC082E94B
:1024D00091E017C084E991E014C081E292E011C05C
:1024E00083E292E00EC084E292E00BC085E292E0CB
:1024F00008C086E292E005C087E292E002C08AE26C
:1025000092E0CF910C947110CF910895882329F116
:102510009CEF980F913A18F40E940C1C0DC090E2A9
:10252000980F983058F4877091E001C0990F8A9500
:10253000EAF7892F0E946A1C0C949E1C9BE5980F59
:10254000933020F480E090E00C944310885A853159
:1025500020F480E090E00C9471100895882321F01D
:102560000E94641C0C949E1C0895882321F00E94F4
:102570006A1C0C949E1C0895BF92CF92DF92EF923A
:10258000FF920F931F93CF93DF9300D000D000D022
:10259000CDB7DEB725E0FC01DE01119601900D926A
:1025A0002A95E1F7FC0140815181028163817481A8
:1025B000258122952F706115710509F403C35F3FD2
:1025C00019F44F3F09F4FEC26C01862F7D836C83A2
:1025D000602F782F8D812E830E943D1B182FB92EDE
:1025E0000E943C1B0E942C1AEB2DE295EF70F0E04C
:1025F000EF59FF4F2E810C94B1268B2D807F9B2DA0
:102600009F70F92E882319F0F29490EFF92200239D
:1026100049F0FF2009F483C28F2D0E94771C0E948D
:102620009E1C7DC2812F0E948612FF2009F4CAC21F
:102630008F2D0E947D1C26960FB6F894DEBF0FBE2C
:10264000CDBFDF91CF911F910F91FF90EF90DF9061
:10265000CF90BF900C949E1C8B2D807F9B2D9F70E4
:10266000F92E803219F0F29480EFF822112319F03C
:10267000113009F12AC00023B1F08F2D222351F12E
:10268000213041F526960FB6F894DEBF0FBECDBFC0
:10269000DF91CF911F910F91FF90EF90DF90CF903E
:1026A000BF900C94871C222319F0213009F48AC2B0
:1026B0000E948A1C2DC00023F1F0263008F082C24F
:1026C0000E94611C8F2129F023C00023F9F0211101
:1026D00016C08F2D26960FB6F894DEBF0FBECDBF65
:1026E000DF91CF911F910F91FF90EF90DF90CF90EE
:1026F000BF900C94AE12253008F064C209C0F601F8
:10270000858180FF0CC28F708583E3CF21111CC2AD
:102710008F2D83C12B2D26952695237030E0211512
:10272000310521F021303105D1F04CC2002321F0D8
:10273000812F9B2D937002C080E090E026960FB60B
:10274000F894DEBF0FBECDBFDF91CF911F910F91E7
:10275000FF90EF90DF90CF90BF900C944310002338
:1027600021F0812F9B2D937002C080E090E026968F
:102770000FB6F894DEBF0FBECDBFDF91CF911F9192
:102780000F91FF90EF90DF90CF90BF900C9471105D
:10279000812F002319F00E94451F02C00E94AD1F27
:1027A00026960FB6F894DEBF0FBECDBFDF91CF9156
:1027B0001F910F91FF90EF90DF90CF90BF900C94FE
:1027C00032208B2D837009F07BC00111FBC1812F5A
:1027D000829586958770880F880F912F9F70C92EDC
:1027E000D12CE12CF12C082E04C0CC0CDD1CEE1CED
:1027F000FF1C0A94D2F714FF12C04FE050E060E0D3
:1028000070E004C0440F551F661F771F8A95D2F7EA
:10281000CB01BA01609570958095909503C060E0FA
:1028200070E0CB012B2D269526952370422F50E08A
:1028300042305105D9F04330510569F16C297D29A9
:102840008E299F294130510551F126960FB6F894F3
:10285000DEBF0FBECDBFDF91CF911F910F91FF90D3
:10286000EF90DF90CF90BF900C94511A6C297D2986
:102870008E299F2926960FB6F894DEBF0FBECDBFD6
:10288000DF91CF911F910F91FF90EF90DF90CF904C
:10289000BF900C946B1A0E94511AC701B60126967C
:1028A0000FB6F894DEBF0FBECDBFDF91CF911F9161
:1028B0000F91FF90EF90DF90CF90BF900C94371A5C
:1028C000002319F08B2D817001C08695882309F4AF
:1028D00079C1812F829586958770880F880F912FF7
:1028E0009F70C92ED12CE12CF12C082E04C0CC0CE9
:1028F000DD1CEE1CFF1C0A94D2F714FF12C04FE03F
:1029000050E060E070E004C0440F551F661F771F61
:102910008A95D2F7CB01BA01609570958095909514
:1029200003C060E070E0CB012B2D26952695237027
:10293000422F50E042305105D9F04330510569F142
:102940006C297D298E299F294130510551F1269608
:102950000FB6F894DEBF0FBECDBFDF91CF911F91B0
:102960000F91FF90EF90DF90CF90BF900C94181BC9
:102970006C297D298E299F2926960FB6F894DEBFF3
:102980000FBECDBFDF91CF911F910F91FF90EF90C0
:10299000DF90CF90BF900C942A1B0E94181BC70198
:1029A000B60126960FB6F894DEBF0FBECDBFDF91FD
:1029B000CF911F910F91FF90EF90DF90CF90BF903C
:1029C0000C94061B103FD1F128F480E4810F803273
:1029D00050F0A0C0123F09F462C008F44BC0133F8E
:1029E00009F472C097C0F12FF071FF2E8B2D8F71FB
:1029F000002351F00E949F1A812FFF2019F0829529
:102A0000807F68CE8F7066CE0E94C01A812FFF2013
:102A100019F08295807F01C08F7026960FB6F894CA
:102A2000DEBF0FBECDBFDF91CF911F910F91FF9001
:102A3000EF90DF90CF90BF900C94B5120023B1F0CF
:102A4000253008F0BFC08B2D8F7126960FB6F894F5
:102A5000DEBF0FBECDBFDF91CF911F910F91FF90D1
:102A6000EF90DF90CF90BF900C94E51A263008F0DD
:102A7000A9C0E9CF0023A9F08B2D8F7126960FB640
:102A8000F894DEBF0FBECDBFDF91CF911F910F91A4
:102A9000FF90EF90DF90CF90BF900C949F1A00238F
:102AA00059F38B2D8F7126960FB6F894DEBF0FBEAB
:102AB000CDBFDF91CF911F910F91FF90EF90DF90ED
:102AC000CF90BF900C94C01A002399F08B2D8F717A
:102AD00026960FB6F894DEBF0FBECDBFDF91CF9123
:102AE0001F910F91FF90EF90DF90CF90BF900C94CB
:102AF0008A1A26960FB6F894DEBF0FBECDBFDF91BF
:102B0000CF911F910F91FF90EF90DF90CF90BF90EA
:102B10000C94851A0023A9F0222309F4ADCF812F4C
:102B200026960FB6F894DEBF0FBECDBFDF91CF91D2
:102B30001F910F91FF90EF90DF90CF90BF900C947A
:102B4000DC11222309F4ADCF812F26960FB6F8941D
:102B5000DEBF0FBECDBFDF91CF911F910F91FF90D0
:102B6000EF90DF90CF90BF900C9486124B2D4F705A
:102B7000612FC6010E94EF1D26960FB6F894DEBFA6
:102B80000FBECDBFDF91CF911F910F91FF90EF90BE
:102B9000DF90CF90BF900C9485194B2D4F70612F13
:102BA000C60126960FB6F894DEBF0FBECDBFDF91EB
:102BB000CF911F910F91FF90EF90DF90CF90BF903A
:102BC0000C94F21D26960FB6F894DEBF0FBECDBF53
:102BD000DF91CF911F910F91FF90EF90DF90CF90F9
:102BE000BF9008950E94841C0E94531C0E949E1C4A
:102BF0000E9464210E94322080E090E00E944310F5
:102C000080E090E00C9471100E94741C0C94F215FA
:102C1000CF93DF9300D000D01F92CDB7DEB7942FB3
:102C20004983252F5A836B837C838D834C815D81FF
:102C3000452B39F12F3F11F49F3F19F149815A81FA
:102C40006B817C818D810E943D1B292F22952F70E5
:102C500030E02C30310504F52A3031055CF4225087
:102C600031092230310568F4853A80F4843090F4DB
:102C7000823080F0883E38F4803E60F48450813A9F
:102C800048F080E014C0803FE1F704C090E2980F64
:102C9000983080F781E00BC02C30310521F493FB94
:102CA000882780F904C02F303105C9F3EACF0F908F
:102CB0000F900F900F900F90DF91CF910895CF93C9
:102CC000DF9300D000D01F92CDB7DEB70F900F90EA
:102CD0000F900F900F90DF91CF910895CF93DF93D6
:102CE00000D000D000D0CDB7DEB726960FB6F8944E
:102CF000DEBF0FBECDBFDF91CF9108951F93CF935D
:102D0000DF93C091CE0116E08091CF01C81799F0F2
:102D1000D0E01C9FF0011D9FF00D1124E053FE4FE9
:102D20004081518162817381848195810E946E16F8
:102D30002196C770E9CFDF91CF911F9108954091FF
:102D40000002509101026091020270910302809191
:102D50000402909105020C946E16809105028295F2
:102D60008F7009F054C080910202882309F44FC08B
:102D70008091CE01A091CF0160910002709101027B
:102D80004091030250910402B6E08A1709F43FC053
:102D900090E041155105C1F17F3F11F46F3FA1F162
:102DA000B89FF001B99FF00D1124E053FE4F21812F
:102DB00072132AC02081621327C02281211124C0EE
:102DC000238134812417350710F421503109241B45
:102DD000350B283C3105C0F4209105022F7020618D
:102DE0002093050226E0289FF001299FF00D112471
:102DF000EB52FE4F80818F708061808380E092E093
:102E00000E94BC120C947E1601968770BECF089566
:102E1000BF92CF92DF92EF92FF920F931F93CF93C7
:102E2000DF93CDB7DEB761970FB6F894DEBF0FBE64
:102E3000CDBF7C0185E0F701DE011D9601900D926A
:102E40008A95E1F7D7014C9111965C9111971296F2
:102E5000DC90129713960D911C91149730910002FB
:102E6000609101028091030290910402009709F49D
:102E700077C16F3F19F43F3F09F472C1B09002026D
:102E8000BB2009F4C5C0209105020817190728F0D6
:102E9000F801E81BF90BCF0104C080959095800FD5
:102EA000911FCC24C394883C910580F0C12C207FD5
:102EB00009F0CCC0702F198B088B6D2D89890E9469
:102EC0005F1680E092E00E94BC12B6C0822F807F25
:102ED00009F047C0651314C0341312C0D11010C0DC
:102EE0002F702061209305020E949F1680E092E0DF
:102EF0000E94BC1280910502D70115968C932FC0B9
:102F00000115110519F15F3F11F44F3FF9F0CD2C78
:102F1000D1101CC08091CE012091CF0136E08217E4
:102F200009F45CC090E0389FF001399FF00D112446
:102F3000E053FE4F6181561306C06081461303C003
:102F40006281611103C001968770E9CFCD2CDD202D
:102F500009F426C180910502816080930502C12C8D
:102F60001FC1651308C0341306C0D11004C080917E
:102F70000502D701C9C04D875E87DF86702F198B88
:102F8000088B6D2D89890E9408168823E9F1DD20C0
:102F9000D9F120910502822F82958F7090E00297DF
:102FA00074F0809100029091010298878F831986B6
:102FB0001B870A872C87CE0107960E94BC1286E0E9
:102FC000F701A0E0B2E001900D928A95E1F70E942E
:102FD000AD160E949F16CC24C394E2C0702F198BAB
:102FE000088B60E089890E943D1B292F22952F7054
:102FF00030E0223031050CF0C7C09F7009F0C1C02D
:10300000805E883008F4CCC0C7010E94BC12E3CFB8
:103010000817190708F456C0F801E81BF90BCF018F
:10302000883C910508F453C0C12C702F198B088B74
:103030006D2D89890E945F16E0E0F2E086E0DF01F5
:103040001D928A95E9F70E949F16AAC0651314C0C5
:10305000341312C0D11010C080910502F70185838E
:10306000C7010E94BC1286E0E0E0F2E0DF011D92A1
:103070008A95E9F7CB2C94C04D875E87DF86702F49
:10308000198B088B6D2D89890E940816882309F4F5
:10309000BBCFDD2009F4B8CF20910502822F8295A5
:1030A0008F7090E002970CF48ACF8091000290918B
:1030B00001029A8389831B821D830C832E83CE0198
:1030C00001967BCF80959095800F911FA9CFCD2C35
:1030D000DD2009F499CF65132EC034132CC0209144
:1030E000050220FD1FC0822F82958F70D9F0D70175
:1030F00015962C9315978F3049F08F5F982F9295E6
:10310000907F822F8F70892B15968C93C7010E9418
:10311000BC1286E0F701A0E0B2E001900D928A9522
:10312000E1F791CF86E0F701A0E0B2E001900D92C7
:103130008A95E1F735C04D875E87DF86702F198B42
:10314000088B6D2D89890E940816811138CF8091D6
:103150000502816080930502C7010E94BC1220C055
:10316000DD2009F451CF4D875E87DF86702F198BE4
:10317000088B6D2D89890E940816882309F444CF95
:103180001ECF81113DCF0CC0243031050CF03CCF57
:103190009F7009F435CFF7019581907F09F030CF0A
:1031A0008C2D61960FB6F894DEBF0FBECDBFDF91B8
:1031B000CF911F910F91FF90EF90DF90CF90BF9034
:1031C00008951F93CF93DF93CDB7DEB72C970FB63B
:1031D000F894DEBF0FBECDBF4F83588769877A87CB
:1031E0008B879C87CE0107960E940817882369F079
:1031F0008F8198852A853B85232BF1F19F3F09F02C
:1032000063C08F3F09F060C037C086E0FE0137968B
:10321000DE01119601900D928A95E1F76F81788514
:10322000EA85FB85309741F17F3F11F46F3F21F133
:103230002091CF0130E0C901019687709927409114
:10324000CE0150E08417950709F447C069837A835B
:10325000FD83EC8396E0929FD001939FB00D1124E3
:10326000A053BE4FFE01319601900D929A95E1F761
:103270008093CF010E947E1616E08091CE0190913E
:10328000CF018917C1F1189FC001112480539E4FAF
:103290000E940817882379F1E091CE011E9FF0016A
:1032A0001124E053FE4F40815181628173818481FA
:1032B00095810E946E168091CE0190E001968770F4
:1032C00099278093CE01D9CF4F81588569857A851A
:1032D0008B859C850E946E16CFCF0E94041610929B
:1032E000CF011092CE01E0E0F2E086E0DF011D9216
:1032F0008A95E9F7C1CF2C960FB6F894DEBF0FBEC2
:10330000CDBFDF91CF911F910895DF92EF92FF9291
:103310000F931F93CF93DF93FC01892B09F48AC08D
:10332000E12CF12CDD24D394EF0121968491853793
:1033300009F461C058F4843708F04EC0843008F0B6
:103340006AC08130D1F0823071F174C0883709F4DD
:103350005DC050F4863709F455C0873709F06AC05C
:103360008E2D0E94711C54C09CE7980F903708F076
:1033700061C08F770E94861250C08F010E5F1F4F71
:10338000FE01849190E2980F983050F48770FD2DE3
:1033900001C0FF0F8A95EAF78F2F0E94771C14C097
:1033A0000E94DC1113C08F010E5F1F4FFE01C491FC
:1033B00080E28C0F883060F4C7708D2D01C0880FBB
:1033C000CA95EAF70E947D1C0E949E1CE80125C058
:1033D0008C2F0E948612FACF9F012E5F3F4FFE0175
:1033E000C491CC2369F08FE99FE00197F1F700C009
:1033F0000000C150F6CF9F012E5F3F4FFE01F490B9
:10340000E9010BC00E94611CE82E07C00E94741CD9
:103410000E949E1C02C00E94DC118F2D882341F067
:10342000EFE9FFE03197F1F700C000008150F6CFDF
:10343000FE017ACFDF91CF911F910F91FF90EF9016
:10344000DF900895609386027093870280938802CC
:10345000909389020C94F01C089560938A027093F3
:103460008B0280938C0290938D020C94EF1C0F932F
:103470001F9300918A0210918B0220918C0230914F
:103480008D02602B712B822B932B60938A02709399
:103490008B0280938C0290938D021F910F910C945C
:1034A000EF1C0F931F9300918A0210918B022091C1
:1034B0008C0230918D0260237123822393236093C9
:1034C0008A0270938B0280938C0290938D021F91DD
:1034D0000F910C94EF1C0F931F9300918A0210918F
:1034E0008B0220918C0230918D02602771278227F8
:1034F000932760938A0270938B0280938C0290933F
:103500008D021F910F910C94EF1C60E070E0CB01D5
:103510000C94221A0F931F9341E050E060E070E09A
:103520008A019B0104C0000F111F221F331F8A95BF
:10353000D2F7C901B8011F910F910C94221A0F9371
:103540001F9341E050E060E070E004C0440F551F5D
:10355000661F771F8A95D2F7809186029091870225
:10356000A0918802B09189028A019B01082B192B36
:103570002A2B3B2BC901B8011F910F910C94221AE1
:103580000F931F9341E050E060E070E004C0440FEF
:10359000551F661F771F8A95D2F740955095609505
:1035A00070958091860290918702A0918802B091D7
:1035B00089028A019B01082319232A233B23C9017D
:1035C000B8011F910F910C94221A0F931F9341E0A1
:1035D00050E060E070E004C0440F551F661F771F85
:1035E0008A95D2F78091860290918702A0918802F5
:1035F000B09189028A019B01082719272A273B27B6
:10360000C901B8011F910F910C94221A0F931F93B7
:1036100000918602109187022091880230918902E0
:10362000602B712B822B932B1F910F910C94221ADC
:103630000F931F93009186021091870220918802B8
:103640003091890260237123822393231F910F916C
:103650000C94221A0F931F930091860210918702F7
:103660002091880230918902602771278227932751
:103670001F910F910C94221A08958F929F92AF92EE
:10368000BF92DF92EF92FF920F931F93CF93DF933E
:1036900000D000D01F92CDB7DEB76B837C838D83C3
:1036A0008A018C819D81892B21F01F3F29F44F3F96
:1036B00019F480E090E04CC08B818823C9F18090A0
:1036C0008A0290908B02A0908C02B0908D02809123
:1036D000860290918702A0918802B0918902882A7F
:1036E000992AAA2ABB2A8FE1E82EF12CD501C40120
:1036F0000E2C04C0B695A795979587950A94D2F796
:1037000080FF07C0DE2CB8018E2D0E940E1E01978F
:1037100029F481E0E81AF10848F7D12C88E0189FD5
:10372000F0011124E00FF11DEA5FFD4FD08209C0C6
:1037300088E0189FF0011124E00FF11DEA5FFD4FB2
:10374000D08009831A8369817A818D2D0E940E1E93
:103750000F900F900F900F900F90DF91CF911F91CE
:103760000F91FF90EF90DF90BF90AF909F908F9060
:10377000089590910A01992321F090910B019111E4
:1037800009C020910C0130910D01F90132969FEF93
:1037900040E030C0982F9695969596959F31A0F46D
:1037A000E0910C01F0910D01E90FF11D877021E00E
:1037B00030E0A90102C0440F551F8A95E2F7CA0103
:1037C0009181892B818308959091B10290FF23C04C
:1037D0001F928F938BE194E09F938F930E94270613
:1037E0000F900F900F900F9008959F3F39F04F5F0B
:1037F0004E3141F051915813F8CF0DC05111F7CF10
:10380000942FF5CF9F3F39F0F901E90FF11D97FD96
:10381000FA9582830895089590910A01992321F0E1
:1038200090910B01911109C020910C0130910D0173
:10383000F9013296205E3F4F30C0982F96959695AD
:1038400096959F31A8F4E0910C01F0910D01E90FDC
:10385000F11D877021E030E0A90102C0440F551F1F
:103860008A95E2F7CA018095918189238183089521
:103870009091B10290FF16C01F928F938DEF93E04D
:103880009F938F930E9427060F900F900F900F9099
:1038900008953196E217F30729F090819813F9CF34
:1038A0001082F7CF089581E090E0E0910C01F09153
:1038B0000D01E80FF91F1082019680329105A9F7DA
:1038C00008958091B00208959091B002892B809361
:1038D000B002089580959091B00289238093B00240
:1038E00008958093B00208951092B00208959091C7
:1038F000AF02892B8093AF02089580959091AF021B
:1039000089238093AF0208951092AF0208958093A7
:103910008E02089510928E02089580910C0190916C
:103920000D01FC0131969C01205E3F4F80E091919A
:1039300091118F5FE217F307D1F70895E0910C0121
:10394000F0910D018091B0028083E0910C01F09123
:103950000D0190818091AF02892B808380918E022E
:10396000882361F0E0910C01F0910D019081892B89
:1039700080830E948D1C811110928E0280910C0117
:1039800090910D010C94EF0F9093390180933801C1
:1039900008958295982F9C7C392F36953695282F3F
:1039A000237344E0249FC0011124932F982B292FC7
:1039B0002A7A2695892F8575880F822B0895089578
:1039C000CF93DF9300D000D01F92CDB7DEB70F901A
:1039D0000F900F900F900F90DF91CF910895089561
:1039E00008950C9448118091C602843021F1109200
:1039F000B20220E488E190E00FB6F894A895809395
:103A000060000FBE2093600083B7817F846083BF16
:103A100083B7816083BF7894889583B78E7F83BF97
:103A20000FB6F894A895809160008861809360003B
:103A3000109260000FBE0895CF930E949A110E94C9
:103A400077070E949B11C0E08C2F0E94FE07811116
:103A500004C0CF5FC031C1F701C081E0CF910895AC
:103A60000E9404080C9404161F920F920FB60F9236
:103A700011248F939F93AF93BF938091B2028111D2
:103A800013C08091B3029091B402A091B502B0919D
:103A9000B6024196A11DB11D8093B3029093B4026A
:103AA000A093B502B093B602BF91AF919F918F9151
:103AB0000F900FBE0F901F90189582E084BD93E089
:103AC00095BD9AEF97BD80936E0008952FB7F89437
:103AD0008091B3029091B402A091B502B091B60268
:103AE0002FBF08952FB7F8946091B3027091B4027C
:103AF0008091B5029091B6022FBF0895CF92DF92C8
:103B0000EF92FF920F931F932FB7F8944091B30257
:103B10005091B4026091B5027091B6022FBF6A0154
:103B20007B01EE24FF248C0120E030E0C016D1069A
:103B3000E206F30610F4415051099A01281B390B93
:103B4000C9011F910F91FF90EF90DF90CF900895E2
:103B50001F920F920FB60F9211248F939F93AF93E2
:103B6000BF938091B3029091B402A091B502B0913D
:103B7000B6020196A11DB11D8093B3029093B402C9
:103B8000A093B502B093B602BF91AF919F918F9170
:103B90000F900FBE0F901F9018950E94F10CF89493
:103BA0002FEF87EA91E6215080409040E1F700C076
:103BB000000087E090EBDC018093CF029093D0026D
:103BC000A093D102B093D2029CE088E10FB6F894A2
:103BD000A895809360000FBE90936000FFCF80E0B7
:103BE00090E008950895E72FF0E090E1899FE00DBF
:103BF000F11D112483E0EE0FFF1F8A95E1F7E60F18
:103C0000F11DEE51FF4F84910895E82FF0E0EE0F83
:103C1000FF1FEE59F0408591949108950E94F31D85
:103C200090E4980F903218F40E94051E08958D3B81
:103C300050F4883AA0F5853A28F5843000F58130B3
:103C400009F49DC099C0883E98F4803EC0F48F3B33
:103C500009F092C00E9404162FEF80E792E02150F5
:103C600080409040E1F700C000000E94CD1D84C05C
:103C7000803F08F481C0282F30E0306582C0282FB3
:103C800030E07FC0853A29F0863A31F023E830E40D
:103C900078C021E830E475C022E830E472C0883A88
:103CA00061F1893A69F18A3A71F18B3A79F18C3A8A
:103CB00081F18D3A89F18E3A91F18F3A99F1813BF8
:103CC000A1F1803BA9F1823BB1F1833BB9F1843B87
:103CD000C1F1853BC9F1863BD1F1873BD9F1883BE6
:103CE000E1F1893BE9F18A3BF1F18B3BF9F18C3B46
:103CF00009F43FC020E034E444C022EE34E441C083
:103D000029EE34E43EC02AEE34E43BC025EB34E433
:103D100038C026EB34E435C023EB34E432C024EB66
:103D200034E42FC027EB34E42CC02CEC34E429C05D
:103D30002DEC34E426C023E835E423C02AE835E43A
:103D400020C022E935E41DC024E935E41AC021E28F
:103D500036E417C023E236E414C024E236E411C08E
:103D600025E236E40EC026E236E40BC027E236E454
:103D700008C02AE236E405C020E030E002C021E0BD
:103D800030E0C90108958091B90280FF0BC06091B5
:103D9000110185E0689FB0011124759567957595AF
:103DA00067952BC081FF09C06091110185E0689F74
:103DB000B00111247595679520C082FF07C06091FE
:103DC000110185E0689FB001112417C09091BA02DB
:103DD0009923D1F060911001961788F72091110175
:103DE00085E0289F90011124929FA001939F500D80
:103DF000112470E0CA010E949D266038710540F4CC
:103E00006115710539F002C065E070E0862F0895F4
:103E10008FE7089581E008958091B90280FF08C07E
:103E200060910F0170E0759567957595679521C054
:103E300081FF06C060910F0170E07595679519C00C
:103E400082FF04C060910F0170E010C09091BA022F
:103E50009923C1F060910E019617A0F780910F0190
:103E6000899FC001112470E00E949D266038710571
:103E700028F46115710521F0862F08958FE70895C4
:103E800081E0089561E070E0F4CF803F21F40E946A
:103E9000C31E819504C0813F29F40E94C31E8093F4
:103EA000BD020895823F21F40E94C31E819504C083
:103EB000833F29F40E94C31E8093BC020895893F6A
:103EC00019F40E940C1F05C08A3F31F40E940C1F98
:103ED00081958093BE0208958B3F21F40E940C1FB0
:103EE000819504C08C3F29F40E940C1F8093BF026F
:103EF0000895843F21F48091BB02816017C0853F03
:103F000021F48091BB02826011C0863F21F4809130
:103F1000BB0284600BC0873F21F48091BB028860A4
:103F200005C0883F31F48091BB0280618093BB0261
:103F300008958D3F21F48091B90281600BC08E3FBE
:103F400021F48091B902826005C08F3F29F48091ED
:103F5000B90284608093B9020895803F39F480915A
:103F6000BD0287FF6CC01092BD0269C0813F29F479
:103F70008091BD021816BCF362C09091BC02823FD2
:103F800029F497FF5CC01092BC0259C0833F19F41A
:103F90001916CCF354C0893F41F48091BE02181623
:103FA0000CF04DC01092BE024AC08A3F29F48091A5
:103FB000BE0287FF44C0F6CF8B3F39F48091BF0229
:103FC00087FF3DC01092BF023AC08C3F29F4809118
:103FD000BF021816BCF333C0843F21F48091BB02AA
:103FE0008E7F17C0853F21F48091BB028D7F11C069
:103FF000863F21F48091BB028B7F0BC0873F21F469
:104000008091BB02877F05C0883F31F48091BB025D
:104010008F7E8093BB0213C08D3F21F48091B90243
:104020008E7F0BC08E3F21F48091B9028D7F05C039
:104030008F3F29F48091B9028B7F8093B9028091E0
:10404000BC0281110EC08091BD0281110AC0809115
:10405000BE02811106C08091BF02811102C0109280
:10406000BA0208958091B10283FF7EC080E694E099
:104070000E948E058091BB021F928F938BE594E086
:104080009F938F930E94270689E594E00E948E05F6
:104090008091BC02282F082E000C330B3F938F9386
:1040A00086E594E09F938F930E94270684E594E031
:1040B0000E948E058091BD02282F082E000C330B24
:1040C0003F938F9381E594E09F938F930E942706FF
:1040D0008FE494E00E948E058091BE02282F082E66
:1040E000000C330B3F938F938CE494E09F938F935A
:1040F0000E9427068AE494E00E948E058091BF0208
:10410000282F082E000C330B3F938F9387E494E005
:104110009F938F930E94270684E494E00E948E056B
:104120008091BA021F928F9381E494E09F938F93C2
:104130000E9427068FE394E00E948E058091B902C9
:104140001F928F938CE394E09F938F930E94270696
:1041500089E394E00E948E058DB79EB74C960FB60A
:10416000F8949EBF0FBE8DBF8BEB92E00E9438107B
:104170000E94661D9093B8028093B70208951F9322
:10418000CF93DF938091B7029091B8020E947E1D79
:10419000AC019091BA02992321F02091120130E0F4
:1041A00006C0209113018AE0289F90011124421734
:1041B000530708F485C08091BC02C091BD02D09124
:1041C000BE021091BF02811107C0C11175C0D1118B
:1041D00073C0111171C074C09F3F19F09F5F90931D
:1041E000BA02181624F40E94C31E8093BC02809168
:1041F000BC0287FF05C00E94C31E81958093BC024C
:104200001C1624F40E94C31E8093BD028091BD023F
:1042100087FF05C00E94C31E81958093BD026091F7
:10422000BC02662331F1C091BD02CC2311F1062EF0
:10423000000C770B880B990B0E94982523E333E33E
:1042400043E35FE30E94FC250E9460256093BC026B
:104250006C2FCC0F770B880B990B0E94982523E3CA
:1042600033E343E35FE30E94FC250E9460256093F3
:10427000BD021D1624F40E940C1F8093BE02809183
:10428000BE0287FF05C00E940C1F81958093BE026D
:10429000111624F40E940C1F8093BF028091BF026C
:1042A00087FF05C00E940C1F81958093BF02DF919C
:1042B000CF911F910C9432209F3F09F08FCF97CF61
:1042C000DF91CF911F910895EBEBF2E085E0DF01E4
:1042D0001D928A95E9F71092BA021092B9020895D8
:1042E00083E896E00E948E051F9281E08F931F92D3
:1042F00085E08F9385E396E09F938F930E94270636
:104300000F900F900F900F900F900F9008958330A3
:10431000E9F128F4813061F0823009F108958530A7
:1043200009F462C008F449C0863009F474C00895E5
:1043300080911301262F30E0280F311D2F3F3105CA
:1043400024F4680F6093130103C08FEF809313016F
:10435000809113011F928F938EE695E072C0809139
:104360001201262F30E0280F311D2F3F310524F494
:10437000680F6093120103C08FEF80931201809148
:1043800012011F928F938CE595E05BC08091110123
:10439000262F30E0280F311D2F3F310524F4680F00
:1043A0006093110103C08FEF80931101809111017F
:1043B0001F928F9389E495E044C080911001262FCD
:1043C00030E0280F311D2F3F310524F4680F609332
:1043D000100103C08FEF80931001809110011F9294
:1043E0008F9384E395E02DC080910F01262F30E05C
:1043F000280F311D2F3F310524F4680F60930F0102
:1044000003C08FEF80930F0180910F011F928F9354
:104410008BE195E016C080910E01262F30E0280F29
:10442000311D2F3F310524F4680F60930E0103C046
:104430008FEF80930E0180910E011F928F9380E089
:1044400095E09F938F930E9427060F900F900F90F7
:104450000F900895833081F128F4813059F0823033
:10446000D1F00895853009F449C0B8F1863009F4D7
:1044700056C0089580911301681720F4861B80931D
:10448000130102C010921301809113011F928F93A8
:1044900081EF94E054C080911201681720F4861BCC
:1044A0008093120102C010921201809112011F929A
:1044B0008F938FED94E043C080911101681720F431
:1044C000861B8093110102C010921101809111018D
:1044D0001F928F938CEC94E032C08091100168178A
:1044E00020F4861B8093100102C01092100180916D
:1044F00010011F928F9387EB94E021C080910F01F0
:10450000681720F4861B80930F0102C010920F01E0
:1045100080910F011F928F938EE994E010C08091DB
:104520000E01681720F4861B80930E0102C01092C2
:104530000E0180910E011F928F9383E894E09F9368
:104540008F930E9427060F900F900F900F90089561
:10455000CF93C82F1F928F9388E897E09F938F93F4
:104560000E94270681E090E0A0E0B0E0BC01CD0110
:1045700004C0660F771F881F991FCA95D2F70E9443
:104580002D1A0F900F900F900F90CF910C9404164E
:10459000CF938732A8F58E3108F02BC1803109F412
:1045A0009FC0F8F4873009F464C0A8F4863009F09D
:1045B00024C18091B102817F8E7F8093B1028DE80A
:1045C00097E00E948E058AE69AE00E948E0581E0BF
:1045D0008093C1024CC08B30F1F18E3009F46CC075
:1045E0000CC1863109F4B0C020F4813109F4EDC06A
:1045F00004C1893109F491C08B3109F449C0FDC06F
:10460000883349F150F4893209F4F1C0853309F453
:10461000EEC0873209F0F1C0EAC0833409F4E7C084
:1046200028F48A3308F4E9C08953E4C0883409F0D7
:10463000E4C00E94041689E59AE00E948E052FEFDF
:1046400083ED90E3215080409040E1F700C00000EE
:104650000E94CD1D0CC084EB97E05CC080E49AE022
:104660000E948E058091B10281608093B102C1E009
:10467000C9C08091B102C82FC17080FFEFCF8CE418
:104680009AE00E948E058091B102817F8E7F3DC0AD
:104690009091B10291FBCC27C0F981E0C827892F06
:1046A000C0FB81F98093B102CC2319F083E39AE037
:1046B00027C085E29AE02EC09091B10292FBCC27F0
:1046C000C0F981E0C827892FC0FB82F98093B1022D
:1046D000CC2319F086E19AE013C086E09AE01AC074
:1046E0009091B10293FBCC27C0F981E0C827892FB4
:1046F000C0FB83F98093B102CC2351F08AEF99E09B
:104700000E948E058091B10281608093B1027AC0CF
:104710008DEE99E00E948E05AACF8EED99E00E9461
:104720008E058CEB99E00E948E0588E799E00E9447
:104730008E058BE499E00E948E0581E199E00E944C
:104740008E0582EE98E0E6CF84ED98E00E948E051B
:104750000E94E30F1F928F938AEB98E09F938F93B1
:104760000E94270680910A011F928F9383EA98E0A6
:104770009F938F930E9427068091B6011F928F937B
:1047800080E998E09F938F930E94270680910B0108
:104790001F928F938DE798E09F938F930E94270637
:1047A0000E94721D9F938F937F936F9386E698E08C
:1047B0009F938F930E9427068DB79EB746960FB69C
:1047C000F8949EBF0FBE8DBF52CF0E940416C091B9
:1047D0000B0181E0C827C0930B01CC2329F08CE5A5
:1047E00098E00E948E050EC081E598E093CF80E0AE
:1047F00001C08D510E94A8223ACF8FE498E00E9418
:104800008E05C0E08C2FCF91089580E0089580E060
:104810000895CF93C82F8091C102813079F020F0A4
:10482000823009F44DC044C1E0910C01F0910D01BA
:1048300080818152823008F03DC108C0E0910C01B6
:10484000F0910D0180818152823060F48C2F0E94A2
:104850000524811104C08C2F0E94C8222FC081E042
:1048600090E02CC08C2F0E940724811126C0C431F7
:10487000E1F070F4CB3081F0C031D1F40E947021AE
:1048800080E897E00E948E0582E08093C10215C007
:10489000C93259F0C83361F48DE897E00E948E0563
:1048A00084E897E00E948E0508C01092C10204C1FE
:1048B0008EE797E00E948E05FFC081E08170FEC008
:1048C000C43228F5CE3108F0C1C0CB30A1F1D0F40C
:1048D000C73009F0D3C08EE18093130182E3809347
:1048E00012018AE08093110184E18093100188E035
:1048F00080930F0188E280930E0184E296E00E948B
:104900008E05BFC0C33149F1C431C1F0B7C0CB344B
:1049100009F4A9C028F4C93289F0C83361F0AEC0E7
:10492000C13509F49EC0C23509F499C0CE3409F0EE
:10493000A5C06AE09EC00E947021A3C08091C00201
:10494000882319F01092C0029CC081E396E00E9477
:104950008E0581E08093C102B1C08BE096E00E9499
:104960008E0589EF95E00E948E05809113011F92BC
:104970008F9386EF95E09F938F930E94270684EF95
:1049800095E00E948E0582EE95E00E948E05809152
:1049900012011F928F938FED95E09F938F930E944A
:1049A00027068DED95E00E948E058EEC95E00E9425
:1049B0008E05809111011F928F938BEC95E09F9350
:1049C0008F930E94270689EC95E00E948E0588EB64
:1049D00095E00E948E05809110011F928F9385EBC8
:1049E00095E09F938F930E94270683EB95E00E94AA
:1049F0008E058EE995E00E948E0580910F011F9231
:104A00008F938BE995E09F938F930E94270689E906
:104A100095E00E948E0582E895E00E948E058091C7
:104A20000E011F928F938FE795E09F938F930E94C3
:104A300027068DE795E00E948E058DB79EB74896B4
:104A40000FB6F8949EBF0FBE8DBF1BC0CE51EC2F8A
:104A5000F0E0E25DFE4F80818093C00212C061E011
:104A600003C061E006C06AE08091C0020E94872115
:104A700008C08091C0020E942A2203C082E296E010
:104A800013C08091C002882369F01F928F938CE13C
:104A900096E09F938F930E9427060F900F900F90A0
:104AA0000F9004C089E196E00E948E0581E006C067
:104AB0001092C10280E002C080E000CFCF91089543
:104AC0000E9467256894B1110C94F62508950E9400
:104AD000DB2588F09F5798F0B92F9927B751B0F090
:104AE000E1F0660F771F881F991F1AF0BA95C9F772
:104AF00014C0B13091F00E94F525B1E008950C94F6
:104B0000F525672F782F8827B85F39F0B93FCCF3A8
:104B1000869577956795B395D9F73EF490958095EE
:104B2000709561957F4F8F4F9F4F0895E89409C00E
:104B300097FB3EF490958095709561957F4F8F4FD0
:104B40009F4F9923A9F0F92F96E9BB279395F695E6
:104B5000879577956795B795F111F8CFFAF4BB0F64
:104B600011F460FF1BC06F5F7F4F8F4F9F4F16C0C8
:104B7000882311F096E911C0772321F09EE8872F52
:104B8000762F05C0662371F096E8862F70E060E00E
:104B90002AF09A95660F771F881FDAF7880F969587
:104BA000879597F9089557FD9058440F551F59F070
:104BB0005F3F71F04795880F97FB991F61F09F3F0A
:104BC00079F087950895121613061406551FF2CF33
:104BD0004695F1DF08C0161617061806991FF1CF83
:104BE00086957105610508940895E894BB276627AA
:104BF0007727CB0197F908950E940F260C94802601
:104C00000E94722638F00E94792620F0952311F038
:104C10000C9469260C946F2611240C94F6250E949E
:104C2000D32570F3959FC1F3950F50E0551F629FF8
:104C3000F001729FBB27F00DB11D639FAA27F00DF5
:104C4000B11DAA1F649F6627B00DA11D661F829F1C
:104C50002227B00DA11D621F739FB00DA11D621F01
:104C6000839FA00D611D221F749F3327A00D611D1E
:104C7000231F849F600D211D822F762F6A2F112400
:104C80009F5750409AF0F1F088234AF0EE0FFF1F33
:104C9000BB1F661F771F881F91505040A9F79E3F8A
:104CA000510580F00C9469260C94F6255F3FE4F3DF
:104CB000983ED4F3869577956795B795F795E795E0
:104CC0009F5FC1F7FE2B880F911D9695879597F9E9
:104CD000089597F99F6780E870E060E008959FEF7E
:104CE00080EC089500240A94161617061806090683
:104CF000089500240A941216130614060506089552
:104D0000092E0394000C11F4882352F0BB0F40F4D9
:104D1000BF2B11F460FF04C06F5F7F4F8F4F9F4F19
:104D20000895991B79E004C0991F961708F0961B07
:104D3000881F7A95C9F78095089597FB072E16F47A
:104D4000009407D077FD09D00E94BA2607FC05D051
:104D50003EF4909581959F4F0895709561957F4F92
:104D60000895EE0FFF1F0024001C0BBE0790F69164
:104D7000E02D0994AA1BBB1B51E107C0AA1FBB1F52
:104D8000A617B70710F0A61BB70B881F991F5A95D7
:104D9000A9F780959095BC01CD010895F894FFCFB7
:104DA0000D08FE08DB08A708730801018F02280818
:104DB000140A321E404D36223965031803E202C040
:104DC000028702FA0113022C024502650200010269
:084DD0000304050607080900B1
:00000001FF
